S31508000000C8090020D9000008E7000008E900000830
S3150800001000000000000000000000000000000000D2
S31508000020000000000000000000000000EB000008CF
S315080000300000000000000000ED0000081D0B00088D
S31508000040F1000008F1000008F1000008F1000008BE
S31508000050F1000008F1000008F1000008F1000008AE
S31508000060F1000008F1000008F1000008F10000089E
S31508000070F1000008F1000008F1000008F10000088E
S31508000080F10000080000000000000000F100000870
S3150800009000000000F1000008F1000008F100000867
S315080000A000000000F1000008F1000008F100000857
S315080000B0F1000008F1000008F10000080000000047
S315080000C00448854600F032F8004800470710000843
S315080000D0C046C046C8090020064880F30888064876
S315080000E0804706480047FEE7FEE7FEE7FEE7FEE72D
S315080000F0FEE70000C8090020210B0008C10000081F
S3150800010030B50B46014600202022012409E00D46A1
S31508000110D5409D4205D31D469540491B2546954029
S3150800012040191546521E002DF1DC30BD064C01253E
S31508000130064E05E0E36807CC2B430C3C9847103481
S31508000140B442F7D3FFF7C0FFC4100008E410000854
S3150800015000F0BCF8FCE7000010B500F07FF80128B5
S3150800016010D0094C207801280CD100F0B7FDA26800
S3150800017061688918FF31F531884203D30020207061
S3150800018000F0C8F810BD0000D000002010B50D4CD6
S315080001900120207000F0A2FDA06000F05FF80128A1
S315080001A00FD0207801280CD100F098FDA26861686C
S315080001B08918FF31F531884203D30020207000F0FA
S315080001C0A9F810BDD000002010B500F087F800F09F
S315080001D071F800F091FD00F0B2FB00F033F8FFF77C
S315080001E0D5FF10BD10B500F071F800F0A1FD00F0C4
S315080001F03FF8FFF7B1FF10BD7047000007480078C9
S31508000200002805D0012805D0022805D0032803D0E8
S31508000210402070470820704700207047DC00002007
S3150800022007480078002805D0012805D0022805D0FF
S31508000230032803D0402070470820704700207047E5
S31508000240DC00002010B500F081FD00F09DFB02499E
S315080002500020087010BD0000DC00002010B5002446
S3150800026000F082FD002800D00124204610BD0000C1
S3150800027008B56946064800F0BDFB012807D10549BF
S315080002800020087068460178014800F075FD08BD31
S31508000290F0000020DC00002010B5054A1278002A7C
S315080002A002D1C9B200F0EEFB00F098FE10BD0000C6
S315080002B0DC00002010B500F001F810BD10B50248AA
S315080002C000F026FB10BD0000B80B000010B500F0CA
S315080002D001F810BD10B500F021FB10BD10B500F0F7
S315080002E001F810BD72B6704762B6704770B504461D
S315080002F0501E0D4686B2002A0AD028782070641C43
S315080003006D1CFFF7E3FF3046761EB6B20028F4D11F
S3150800031070BD000070B500F016FB00282BD0FFF763
S315080003206BFF154881690122920391438161C16976
S31508000330D2009143C16100F0F3FC0121084600F0A8
S3150800034017FB01256D0700F0F6FA0446BF2620784C
S315080003502870641C6D1CFFF7B9FF3046761EB6B2CE
S315080003600028F4D1032000F01FF800F0E4FA4468EE
S31508000370FFF7BAFFA04770BD0010024009490023E5
S315080003800B61C00048618B61052008610869C207D6
S3150800039001D0C003FAD508694008400008618B619E
S315080003A07047000000E000E003490A6892089200DE
S315080003B002430A60704700000000014000B5074983
S315080003C00A6902231A430A614861086940221043F0
S315080003D00861034800F034F800BD00000020024020
S315080003E0FF0F00000248016980221143016170472E
S315080003F000200240F0B50B4E044630690D46012731
S315080004003843306121800F2000F01AF8042807D1FC
S315080004103169280C3943316160800F2000F010F8EB
S31508000420F0BD00000020024003480249416003492C
S31508000430416070472301674500200240AB89EFCD34
S3150800044010B4124B0246D868C00701D001200AE052
S31508000450D868400701D5022005E0D868C00601D54E
S31508000460032000E00420FF21521E491EFDD1012869
S3150800047001D1002AE7D119697724A14319613421EA
S31508000480D960002A00D1052010BC70470020024020
S31508000490F8B50446480A40021646009022681F46E8
S315080004A00D46501C0BD100992046CB054DD19142E3
S315080004B005D0012201605202201DFFF717FF2168AF
S315080004C00098814205D00146204600F01FF9040035
S315080004D03BD02068281A051900982D1DFF30FF30DB
S315080004E002300090FFF7F2FE281B01214902001F87
S315080004F0884222D31648009D844201D1154C0AE051
S315080005001548854202D1124C054604E0204600F003
S3150800051071F9002803D020462946EA0501D00024AF
S3150800052008E002688A4205D0012201605202201DB5
S31508000530FFF7DCFE002C08D0251D307828706D1CCE
S31508000540761C7F1ECED10120F8BD0020F8BD000024
S31508000550800300207C0100200018000810B50A4816
S315080005600068401C04D0084800F044F9002809D067
S3150800057006480068401C04D0044800F03BF90028EF
S3150800058000D0012010BD0000800300207C0100205F
S31508000590F8B5054643480C46411B601E814216D3F2
S315080005A0284600F085F806462819401E00F080F80F
S315080005B0FF2E0CD0FF280AD004460125A64200D9F2
S315080005C00025032E01D3102C03D9002567E000204F
S315080005D0F8BD002D63D037460026FFF777FE0C20BE
S315080005E03146414330480918097AB94204D10C21E9
S315080005F04E4301468E5905E0761CF6B20E2EECD314
S315080006000026F6430027FFF761FE0C2039464143D2
S31508000610254809180A7AA24204D10C214F430146FB
S31508000620CF5905E07F1CFFB20E2FECD30027FF43FE
S3150800063000940024FFF74AFE0C201B49604340182B
S31508000640017A0098814205D10C20444316482018A7
S31508000650406804E0641CE4B20E2CEBD30020381882
S31508000660401E801B80014030040CFFF7DDFE00278A
S31508000670002C12D9FFF72AFE0C48864206D23046CD
S31508000680FFF79CFE042801D0002506E00120800221
S315080006907F1C3618BFB2A742ECD3FFF7A3FE284645
S315080006A0F8BD0000FFFF00081C10000800F0000855
S315080006B070B5054600240C4EFFF708FE21460C20AF
S315080006C041437058A84209D8891949684018A84270
S315080006D004D90C204443A019007A70BD641CE4B206
S315080006E00E2CE9D3FF2070BD1C1000080048704787
S315080006F00018000800200349C04308600249086042
S31508000700704700007C0100208003002070B5044675
S3150800071010480D46844201D10F4C0AE00F48854225
S3150800072002D10C4C054604E0204600F063F8002888
S3150800073004D020462946EA0501D0002070BD02688B
S315080007408A4205D0012201605202201DFFF7CEFD24
S31508000750204670BD800300207C0100200018000898
S315080007600C480B4A43680168591883685918C368C6
S315080007705918036959184369806959184018064970
S3150800078009680818106001D00020704701207047DA
S31508000790E000002000180008C018000870B50446DC
S315080007A010480D46011B681E1646814214D3204682
S315080007B0FFF77EFFFF280FD06019401EFFF778FF6E
S315080007C0FF2809D0600A0849400288422B4632466B
S315080007D0214603D1054802E0002070BD0448FFF712
S315080007E057FE70BDFFFF00080018000880030020B0
S315080007F07C010020F8B50546012000902868FFF71F
S3150800080057FFFF2810D0FFF70FFE00242868A10025
S31508000810461848194768FFF759FD39463046FFF725
S31508000820E9FD042805D101E00020F8BD3068B8428A
S3150800083002D00020009002E0641C802CE6D3FFF76B
S31508000840D1FD0098F8BD000008B5002000900E48BC
S315080008500168491C15D0826841685118C268511848
S3150800086002695118426951188269C06951184018BD
S31508000870C043401C00906A4604210448FFF78EFFD7
S3150800088008BD012008BD000080030020C01800082C
S315080008904B0710B4DB0E082901D2203000E02430C3
S315080008A00F249C4001689A40A1431143016010BC83
S315080008B07047000010B50121880400F04DF8134C6C
S315080008C0032211462046FFF7E3FF032204212046B0
S315080008D0FFF7DEFF21680F200003814321602168AE
S315080008E0E21311432160216A81432162206A0321B0
S315080008F0090308432062206A0F21090488432062FD
S31508000900206A032109040843206210BD0004004838
S315080009100149088070470000CC000020704710B5D8
S31508000920FFF792FF002801D0FFF718FE10BD10B59B
S31508000930FFF72EFE10BD10B5FFF7D8FE10BD10B597
S31508000940FFF7D8FE10BD10B5FFF70AFF10BD10B5AA
S31508000950FFF724FF10BD0000044A0029516901D0A1
S31508000960014300E0814351617047000000100240D6
S31508000970044A0029916901D0014300E0814391614D
S31508000980704700000010024070B5174881690122BF
S31508000990920311438161C1681143C160C1689143E3
S315080009A0C160124CA06940084000A061A0691821E6
S315080009B00843A061E06930210843E0610C48E12161
S315080009C0006849030546FFF79BFB2062E1214902BF
S315080009D02846FFF795FB0007000F6062A069012112
S315080009E00843A06170BD00000010024000380140B5
S315080009F0C8000020F3B5204C844662780025022002
S31508000A001E4F1F4981B0002A19D02378BE68CA181C
S31508000A10521CB60725D57E68167078615B1CDAB25B
S31508000A2022700878904223D16046491CFFF75EFC85
S31508000A306570029821780170012003B0F0BD104A54
S31508000A40B968890714D57968C9B211707861491EE1
S31508000A503F290DD800F042F96060257001206070CA
S31508000A6006E000F03BF961686431884200D9657098
S31508000A70002003B0F0BD0000E4000020003801406B
S31508000A8084050020F3B581B00E46402903D97521A7
S31508000A9019A0FFF75DFB204F3E6000F01FF90446E2
S31508000AA0B8680A34C00708D1FFF710FC00F016F939
S31508000AB0A04202D8B868C007F6D00024002E18D97C
S31508000AC0FFF704FC0198005D386000F007F9054659
S31508000AD0B8680A35C00708D1FFF7F8FB00F0FEF83A
S31508000AE0A84202D8B868C007F6D0641CA4B2B442BB
S31508000AF0E6D303B0F0BD0000536F757263655C4FB3
S31508000B0070656E424C545C706C6174666F726D5C95
S31508000B1072733233322E630000380140704700008A
S31508000B20F0B5634987B00A68012002430A604A683B
S31508000B30604B1A404A600A685F4B1A400A600A68A6
S31508000B4083049A430A604A68C3231B049A434A608B
S31508000B500A685A4B1A400A609F2212048A600A6879
S31508000B6002430A6008688007FCD55648544D564A21
S31508000B70056010681023184310601068C008C0008C
S31508000B80106002200090106802231843106048681D
S31508000B904E4A1040486048689022104348604868AA
S31508000BA04860434841680215114341604848069029
S31508000BB002A8059003A8019000202E460746049037
S31508000BC0F8B2002400900698611C4843791CFFF788
S31508000BD097FAA84201D9401B00E0281A864205D98F
S31508000BE0064605980470019900980870002E08D0EA
S31508000BF0641C402CE7D30498002802D17F1C042FDC
S31508000C00DED3344801698908890001610169490808
S31508000C10490001616946097B254C4907490F01913D
S31508000C206946097A4906490E0091E1698205114328
S31508000C30E1610169284A114001610099019A090494
S31508000C401202114302691143016120680121090654
S31508000C50084320602068800103D400BF2068800113
S31508000C60FBD56068800880006060606802210843E0
S31508000C70606060680007800F022805D000BF6068C2
S31508000C800007800F0228F9D10120FFF777FB61687A
S31508000C901020814361600120FFF770FB60688021A6
S31508000CA0884360600120FFF769FB07B0F0BD0000CC
S31508000CB0001002400CC0FFF8FFFFF6FEFFFF8F0092
S31508000CC000A24A04C8000020002002400FC0FFFF0F
S31508000CD000127A0040100240FFF800FF044800693D
S31508000CE0C103044802D50168491C016000687047C1
S31508000CF000E000E0EC0000200648002101614161A7
S31508000D008161054A426181610522026103480160E9
S31508000D107047000000E000E03F190100EC000020E9
S31508000D2002490020086148618861704700E000E0D8
S31508000D3004480069C00303D503480168491C0160DB
S31508000D407047000000E000E0EC000020044A0021A3
S31508000D50117004489164C170818091705170704718
S31508000D60300100207001002002480078002800D0D9
S31508000D700120704730010020F8B505460078FF26A7
S31508000D80924CFF2810D0924F397801297ED1F42849
S31508000D904CD02CDCD0287AD020DCC92878D0CC28B6
S31508000DA077D0CF2876D1E9E0894D002068700127F1
S31508000DB02F70EE70102129716871FFF71FFAA8715C
S31508000DC0FFF72EFAE871FFF72BFA000A28726F72FE
S31508000DD0AF720820A080FFF7B2FDE2E07C49D12877
S31508000DE08A6C76D0D22875D0F32853D135E0F538F9
S31508000DF00A284FD201007944097949188F44042AF0
S31508000E00CBCBCB4ECB595F6BFFF7F8F96A78401E10
S31508000E1090427DDB381DB96CFFF768FAFE70697879
S31508000E20B86C4018B8646878401CABE0FFF7E6F980
S31508000E306978401E88426BDB6968B9646A78381D30
S31508000E40FFF754FAFE706978B86C4018B864687889
S31508000E50401C97E0FE70686851E05D48C6706F6890
S31508000E60C01D0025164600907F1E07D33078761CD5
S31508000E704019C5B2FFF72AFA7F1EF7D2009801215A
S31508000E800560534801710021417104E09DE039E095
S31508000E9026E079E07FE08171082073E0FE704D4816
S31508000EA0B864002038717871B8714B4807214160E1
S31508000EB0F2E7FE210020F9703871022062E0FE7028
S31508000EC00020387179787971B871F871387206200E
S31508000ED058E04AE03DE0002038707870FE704BE03C
S31508000EE0FFF78CF9411E6A1CB86CFFF730FD002825
S31508000EF029D0FE70FFF782F9B96C401E4018B86415
S31508000F003AE005E0FFF77AF96978801E884205DA43
S31508000F10FE212220F9703871022033E0FE7001208C
S31508000F20A080697800290AD0AA1CB86CFFF70FFDC3
S31508000F30002808D06978B86C4018B86431E0FFF723
S31508000F40EEFC00282DD1FE213120F97038710220DF
S31508000F5018E0FE7000253D717D71FFF74FF9B871F5
S31508000F60FD713D727D7207200CE010466968FFF737
S31508000F70DEFC0028E7D0FE70012003E0FFF7CAF97F
S31508000F80FE700120A0800CE0FE213120F970387136
S31508000F900220A08005E0FE212020F9703871022089
S31508000FA0A080E078012806D10949FE221020CA70DF
S31508000FB008710220A0800421615E002905DD012058
S31508000FC0E070054889B2FFF767F9F8BD700100209F
S31508000FD030010020141000083301002001480021C8
S31508000FE0C17070477001002002E008C8121F08C1CE
S31508000FF0002AFAD170477047002001E001C1121F8C
S31508001000002AFBD17047FFF755FCFFF7DDF8FFF71D
S31508001010E9F8FCE74F70656E424C5400001800086A
S315080010200008000003000000002000080008000077
S315080010300400000000280008000800000500000061
S31508001040003000080008000006000000003800080C
S315080010500008000007000000004000080008000023
S315080010600800000000480008000800000900000009
S3150800107000500008000800000A0000000058000898
S31508001080000800000B0000000060000800080000CF
S315080010900C00000000680008000800000D000000B1
S315080010A000700008000800000E0000000078000824
S315080010B0000800000F000000008000080080000003
S315080010C010000000E4100008C800002028000000F6
S315080010D0E80F00080C110008F0000020D8080000EE
S315080010E0F80F000800A24A040000000000000000F3
S315080010F000000000000000000400000000000000DE
S31108001100000000000000000000000000D5
S705080000C131
